:020000040000FA
:1000000001288312850186018316A83081001F30E4
:100010008500860183128C01803086000F283820ED
:10002000003E03190F2881010C181E288C18232864
:100030000C192A288C1931281D281D28FF30011F72
:10004000030186001E2803308A007F30010500234B
:100050008600252802308A007F30010500228600B4
:100060002C2801308A007F300105002186003328CA
:1000700005183C280C140134851840288C140134D0
:10008000051944280C150134851900348C150134E8
:100200008207FF34FD34FB34F934F734F534F3342A
:10021000F134EF34ED34EB34E934E734E534E334EE
:10022000E134DF34DD34DB34D934D734D534D3345E
:10023000D134CF34CD34CB34C934C734C534C334CE
:10024000C134BF34BD34BB34B934B734B534B3343E
:10025000B134AF34AD34AB34A934A734A534A334AE
:10026000A1349F349D349B3499349734953493341E
:1002700091348F348D348B3489348734853483348E
:1002800081347E347C347A34783476347434723405
:1002900070346E346C346A34683466346434623476
:1002A00060345E345C345A345834563454345234E6
:1002B00050344E344C344A34483446344434423456
:1002C00040343E343C343A343834363434343234C6
:1002D00030342E342C342A34283426342434223436
:1002E00020341E341C341A341834163414341234A6
:1002F00010340E340C340A34083406340434023416
:020300000034C7
:100400008207803486348C34923498349E34A534F8
:10041000AA34B034B634BC34C134C634CB34D0344E
:10042000D534DA34DE34E234E634EA34ED34F03410
:10043000F334F534F834FA34FB34FD34FE34FE344E
:10044000FF34FF34FF34FE34FE34FD34FB34FA3421
:10045000F834F534F334F034ED34EA34E634E2348D
:10046000DE34DA34D534D034CB34C634C134BC3481
:10047000B634B034AA34A5349E34983492348C34D3
:1004800086348034793473346D34673461345A344B
:1004900055344F34493443343E34393434342F34B2
:1004A0002A34253421341D341934153412340F34D0
:1004B0000C340A3407340534043402340134013472
:1004C000003400340034013401340234043405347F
:1004D00007340A340C340F341234153419341D34F3
:1004E000213425342A342F34343439343E344334DF
:1004F00049344F3455345A34613467346D3473346D
:0205000079344C
:100600008207FF34FB34F734F334EF34EB34E73450
:10061000E334DF34DB34D734D334CF34CB34C73492
:10062000C334BF34BB34B734B334AF34AB34A73482
:10063000A3349F349B34973493348F348B34873472
:10064000833480347C347834743470346C3468345B
:10065000643460345C345834543450344C3448344A
:10066000443440343C343834343430342C3428343A
:10067000243420341C341834143410340C3408342A
:1006800004340034043408340C3410341434183472
:100690001C342034243428342C343034343438346A
:1006A0003C344034443448344C345034543458345A
:1006B0005C346034643468346C347034743478344A
:1006C0007C348034833487348B348F349334973440
:1006D0009B349F34A334A734AB34AF34B334B73432
:1006E000BB34BF34C334C734CB34CF34D334D73422
:1006F000DB34DF34E334E734EB34EF34F334F73412
:02070000FB34C8
:02400E00F23F7F
:104200002800430029004600610062007200690036
:10421000630065002000530069006E0063006500C4
:10422000720065002000310037002F00300033009D
:0A4230002F0032003000300037008C
:00000001FF
